:1000000010C017C016C015C014C013C012C011C054
:1000100010C00FC00EC00DC00CC00BC00AC009C07C
:1000200008C011241FBECFE5D1E0DEBFCDBF02D096
:10003000DAC0E6CFBA9AD798CF99D3C0C29A8FE4E4
:1000400093EC0197F1F700C00000C2988FE493ECA5
:100050000197F1F700C00000C29A8FE493EC01977A
:10006000F1F700C00000C2988FE493EC0197F1F71C
:1000700000C00000C29A8FE493EC0197F1F700C032
:100080000000C29A8FE493EC0197F1F700C00000E2
:10009000C2988FE493EC0197F1F700C00000C29A78
:1000A0008FE493EC0197F1F700C00000C2988FE451
:1000B00093EC0197F1F700C00000C29A8FE493EC33
:1000C0000197F1F700C00000C29A8FE493EC01970A
:1000D000F1F700C00000C2988FE493EC0197F1F7AC
:1000E00000C00000C29A8FE493EC0197F1F700C0C2
:1000F0000000C2988FE493EC0197F1F700C0000074
:10010000C29A8FE493EC0197F1F700C00000C29A05
:100110008FE493EC0197F1F700C00000C2988FE4E0
:1001200093EC0197F1F700C00000C29A8FE493ECC2
:100130000197F1F700C00000C2988FE493EC01979B
:10014000F1F700C00000C29A8FE493EC0197F1F739
:1001500000C00000C29A8FE493EC0197F1F700C051
:100160000000C2988FE493EC0197F1F700C0000003
:10017000C29A8FE493EC0197F1F700C00000C29897
:100180008FE493EC0197F1F700C00000C29A8FE46E
:1001900093EC0197F1F700C00000C29A8FE493EC52
:1001A0000197F1F700C00000C2988FE493EC01972B
:1001B000F1F700C00000C29A8FE493EC0197F1F7C9
:1001C00000C00000C2988FE493EC0197F1F700C0E3
:1001D0000000C29A8FE493EC0197F1F700C0000091
:0A01E0002BCFC29829CFF894FFCF6F
:00000001FF
